:020000020000FC
:0200000009C035
:100014000FE90DBF002708BB05E007BB00E407B9E3
:1000240007E806B90FE204BBC09A08E286D0C0987C
:100034001CD0C09A08E281D0C09810D036D0FDCF31
:10004400C09A08E27AD0C09808E277D0F6CF08E2E6
:1000540074D00BD02AD008E270D0FCCF02E453D085
:100064003093600040936100089566240AE0702E86
:1000740001E0802EF3DF09D001E05FD06A94D1F76C
:100084007A94C1F78A94B1F708950091610002301F
:1000940041F400916000073531F0083521F009354D
:1000A40011F0C0980895C09A08950091610003303A
:1000B40040F4023038F0009160000E3618F00A392E
:1000C400A0F00895C09AC29A0AE00F9302E335D0D3
:1000D4000F910A95D1F7C098C2980AE00F9302E3F2
:1000E4002CD00F910A95D1F70895C09AC29A02E3D1
:1000F40024D0C098C29803E10F9302E31ED00F915D
:100104000A95D1F708953327442720E10F9307B9BF
:1001140006B1006406B906B10074E9F704B115B17B
:10012400300F411F0F912A9589F724E08894479551
:1001340037952A95D9F708950EE10F9300E00F93B0
:1001440000E00A95F1F70F910A95C9F70F910A9506
:10015400A1F708950F931F932F933F9300E3002E6D
:10016400102E202E302E402E302F00916100109141
:1001740060002AE3003021F4012F0030C1F000E0D8
:100184000394021671F4032E1394121651F4132ED1
:100194002394221631F4232E3394321611F4332E81
:1001A400439413951A9509F40A951A95E3CF00928E
:1001B40062001092630020926400309265004092C5
:1001C40066003F912F911F910F910895C09A18E0F6
:1001D4000BD0079510F4C09801C0C09A05D01A95A9
:1001E400C1F7C09801D008950F930DEC00000A9553
:0601F400E9F70F910895E8
:00000001FF
